:1000000012C021C020C01FC01EC01DC01CC01BC00C
:100010001AC019C018C017C016C015C014C013C02C
:1000200012C011C010C011241FBECFE5D4E0DEBF46
:10003000CDBF10E0A0E6B0E001C01D92A236B1072E
:10004000E1F729D13EC1DCCFAC9AAC980895282FB6
:1000500080E090E0880F27FF02C0AD9A01C0AD9804
:100060009A998F5FAC9AAC989F5F983011F0220FED
:10007000F1CF0895AB9887EDEADF80E0E8DFAB9A37
:1000800087FFF8CF0895FF920F931F93F82E8B01EF
:10009000F1DFAB9884E8DBDF80E0D9DF812FD7DFA9
:1000A000802FD5DF8F2DD3DFAB9A1F910F91FF905B
:1000B00008950F931F938C01DDDFAB9881EDC7DFAF
:1000C00080E0C5DF812FC3DF802FC1DF80E0BFDF8D
:1000D000AB9A1F910F9108950F931F938C01CADF64
:1000E000AB9888E8B4DFC80126E0969587952A95F5
:1000F000E1F7ADDF802F880F880FA9DF80E0A7DF51
:10010000AB9A1F910F9108950F931F938C01B2DF4B
:10011000AB9883E59CDFC80136E0969587953A95C4
:10012000E1F795DF802F880F880F91DF80E08FDF68
:10013000AB9A1F910F91089520E030E040EA5FE014
:1001400005C0FA013197F1F72F5F3F4F28173907A4
:10015000C0F3089520E040EA5FE0C19AC09880E0D3
:1001600090E0FA013197F1F7019631E08C32930774
:10017000C1F7C198C09A80E090E0FA013197F1F799
:10018000019631E08C329307C1F72F5F253029F7B4
:10019000C198C0980895CF93DF93C19AC09AC0E0E8
:1001A000D0E068DFAB9880E552DFCE0143E0969562
:1001B00087954A95E1F74BDF9E012295220F207E1D
:1001C000822F45DF80E043DFAB9A219634E0C030D8
:1001D000D30739F7C198C09810926100109260005F
:1001E000DF91CF910895CF93DF93C19AC0981DC03E
:1001F00085B1BE0148DF85B182BB219622E0C031C6
:10020000D207B0F3809160009091610065DF80912A
:10021000600090916100019690936100809360006E
:10022000B59B06C08550904218F4C0E0D0E0E6CF00
:100230001092610010926000C198C098DF91CF9138
:100240000895CF93DF93C198C09A809160009091F8
:1002500061005ADFC0E0D0E0CE012BDF82BB2196E7
:1002600022E0C031D207C1F7809160009091610017
:1002700001969093610080936000B59B03C0855008
:10028000904218F31092610010926000C198C098DB
:10029000DF91CF91089583E087BB88EF84BB8FEF18
:1002A00081BB8CE388BB80E287B982EE86B952DFDE
:1002B000B29B71DFB39B97DFB49BC3DF85B182BB79
:0602C000F7CFF894FFCF18
:00000001FF
